:100000000C94D2010C94FA010C94FA010C94FA01AC
:100010000C94FA010C94FA010C94FA010C94FA0174
:100020000C94FA010C94FA010C94FA010C946522D8
:100030000C94FA010C94FA010C94FA010C94FA0154
:100040000C9467240C94FA010C942B270C945D27D4
:100050000C94FA010C94FA010C94FA010C94FA0134
:100060000C94FA010C94FA01C61BB21BB71BB61B09
:10007000BB1BBF1BC11BC51BE61BED1BF41BFB1BE6
:10008000021C191C091C191C101C891C8D1C911C9C
:10009000951C991C9D1CA11C6D61784C656E677444
:1000A000683A20004669727374207761766520682B
:1000B000616C66004D53472C492C596F7520707246
:1000C0006F6261626C7920776F6E27742067657448
:1000D00020616E792064657461696C20696E20749A
:1000E0006869732E0020697320002C20726F77538B
:1000F000697A653A20004D53472C492C4D61782090
:1001000064656E7369747920666F722070656E53D2
:10011000697A653A2000506F776572696E6720646E
:100120006F776E2E004C696E65206973206E6F7458
:10013000206F6E2074686520706167652E20536B98
:10014000697070696E672069742E00546869732045
:10015000706F696E742066616C6C73206F75747358
:10016000696465207468652061726561206F66202E
:1001700074686973206D616368696E652E20536BC6
:10018000697070696E672069742E006D6D00436838
:10019000616E6765642050656E20776964746820BD
:1001A000746F20004E657720616363656C3A2000B0
:1001B0004E6577206D61782073706565643A200024
:1001C000504753504545442C0050474C4946542C09
:1001D000005047535445504D554C5449504C494597
:1001E000522C005047535445505350455252455697
:1001F0002C0050474D4D5045525245562C0050470B
:1002000053495A452C002900706167654865696744
:10021000687420696E2073746570732028005265BD
:1002200063616C6320002900526563616C63207018
:10023000616765576964746820696E2073746570BE
:10024000732028002900292C207374657073506571
:10025000724D4D202800526563616C63206D6D50B6
:100260006572537465702028004C6F61646564206A
:1002700073746570206D756C7469706C6965723A21
:10028000004C6F6164656420757020706F733A0074
:100290004C6F6164656420646F776E20706F733A91
:1002A000004C6F61646564207374657073207065C1
:1002B00072207265763A004C6F61646564206D6DE2
:1002C0005065725265763A004C6F616465642068CF
:1002D00065696768743A004C6F616465642077698A
:1002E0006474683A00206E6F74207265636F676E85
:1002F000697365642E0052454144590029206E6F90
:1003000074207061727365642E00436F6D6D2028D8
:1003100000000000080002010000030407000000C4
:1003200000000000000102040810204080010204C7
:10033000081020010204081020040404040404042A
:10034000040202020202020303030303030000008B
:1003500000250028002B0000000000240027002AB0
:10036000004E414E494E495459494E46CDCCCC3DA4
:100370000AD7233C17B7D13877CC2B329595E62492
:100380001FB14F0A000020410000C84200401C4637
:1003900020BCBE4CCA1B0E5AAEC59D74880DD51B21
:1003A0008D27660E11241FBECFEFD8E0DEBFCDBF74
:1003B00012E0A0E0B1E0E2EDF7E602C005900D9298
:1003C000AA32B107D9F724E0AAE2B2E001C01D9237
:1003D000A03BB207E1F713E0C2EAD3E004C02297E2
:1003E000FE010E94A72ECC39D107C9F70E94AE2B7F
:1003F0000C94DC330C94000043E061E080EC92E06C
:100400000C94001B43E062E080EC92E00C94001B33
:1004100043E061E084EB92E00C94001B43E062E077
:1004200084EB92E00C94001BCF92DF92EF92FF924C
:100430000F931F93CF93DF93CDB7DEB7BC01EDB61B
:10044000FEB6FC0101900020E9F73197E81BF90B9B
:100450008DB79EB78E1B9F0B0FB6F8949EBF0FBE35
:100460008DBF0DB71EB70F5F1F4FC8010E94963199
:100470006CEE71E0C8010E947F318C011092A603DE
:100480001092980310928A0310927C03D12CC12CF5
:10049000D11004C0B80184EB93E03CC06CEE71E075
:1004A00080E090E00E947F318C01009741F0BC0118
:1004B00087EE91E00E94AB31892B09F4C39492E05E
:1004C000D916A1F09D1520F081E0D81641F024C086
:1004D00093E0D91691F084E0D816B1F01DC0011553
:1004E0001105D1F0B80186EA93E014C00115110599
:1004F00099F0B80188E993E00DC00115110561F08C
:10050000B8018AE893E006C00115110529F0B80189
:100510008CE793E00E949631D39496E0D912B8CF3D
:10052000C0927B030FB6F894FEBE0FBEEDBEDF9106
:10053000CF911F910F91FF90EF90DF90CF90089592
:10054000CF93DF93EC0167EE71E00E94AB31FC01C9
:10055000148267EE71E00E948D31892B29F4CE015F
:100560000E94140281E001C080E0DF91CF910895E4
:1005700066EF72E08DE094E00C944C28CF93DF930B
:10058000EC0161E171E08DE094E00E943F28BE0142
:100590008DE094E00E94312865EE72E08DE094E0F9
:1005A000DF91CF910C944C288F929F92AF92BF9283
:1005B000CF92DF92EF92FF928090390190903A01B2
:1005C000A0903B01B0903C01A0913D01B0913E0153
:1005D0002091380130E00E94BA2E0E94C22C6B019B
:1005E0007C019B01AC01C501B4010E94272C6093E2
:1005F000CE037093CF038093D0039093D103A501D2
:100600009401C701B6010E94272C6093CA0370931E
:10061000CB038093CC039093CD0364EF71E080E033
:1006200090E0FF90EF90DF90CF90BF90AF909F90C1
:100630008F900C94E024CF93DF93C0E0D0E04AE0A9
:1006400050E0BE018DE094E00E94132964E571E062
:100650008DE094E00E943F28CE010E9409324AE0DA
:1006600050E0682F8DE094E00E9459292196C8320D
:10067000D10529F7DF91CF91089584E190E00E94A0
:100680000932811101C081E08093380169E672E08E
:100690008DE094E00E940E284AE050E0609138011D
:1006A0008DE094E00C9459290E941B036EEF71E0D9
:1006B0008DE094E00E940E28609136017091370120
:1006C0004AE050E08DE094E00E9413296CEE71E066
:1006D0008DE094E00E943F286091340170913501D3
:1006E0004AE050E08DE094E00E94132967EE71E04B
:1006F0008DE094E00E945E2862EF71E08DE094E06E
:100700000E940E284091390150913A0160913B01BD
:1007100070913C0122E030E08DE094E00E945B2A81
:1007200067EE71E08DE094E00E945E2863EE71E078
:100730008DE094E00E940E2860913D0170913E0191
:100740004AE050E08DE094E00E94132967EE71E0EA
:100750008DE094E00E945E2861ED71E08DE094E010
:100760000E940E284AE050E0609138018DE094E04C
:100770000E94522967EE71E08DE094E00E945E28AD
:1007800069EC71E08DE094E00E940E2860913F01D9
:10079000709140014AE050E08DE094E00E941329FE
:1007A0006CEE71E08DE094E00E943F286091410181
:1007B000709142014AE050E08DE094E00E941329DC
:1007C00067EE71E08DE094E00E945E2860EC71E0DD
:1007D0008DE094E00E940E2840913001509131014B
:1007E000609132017091330122E030E08DE094E0BD
:1007F0000E945B2A6CEE71E08DE094E00E943F283D
:1008000040912C0150912D0160912E0170912F018A
:1008100022E030E08DE094E00E945B2A67EE71E018
:100820008DE094E00C945E28AB01BC014093300154
:1008300050933101609332017093330180E792E06D
:100840000E941F214091300150913101609132018D
:10085000709133018CE292E00E941F2160EB71E005
:100860008DE094E00E940E284091300150913101BA
:10087000609132017091330122E030E08DE094E02C
:100880000C945D2AAB01BC0140932C0150932D01C7
:1008900060932E0170932F0180E792E00E948421E3
:1008A00040912C0150912D0160912E0170912F01EA
:1008B0008CE292E00E94842164EA71E08DE094E091
:1008C0000E940E2840912C0150912D0160912E0123
:1008D00070912F0122E030E08DE094E00C945D2ACD
:1008E00086EA93E00E942E316093250170932601E1
:1008F00080932701909328016EE871E08DE094E0E9
:100900000E940E28409125015091260160912701F7
:100910007091280122E030E08DE094E00E945B2A93
:100920006BE871E08DE094E00C944C284F925F925C
:100930006F927F928F929F92AF92BF92CF92DF92EF
:10094000EF92FF920F931F93CF93DF93CDB7DEB754
:1009500028970FB6F894DEBF0FBECDBF6D837E83A0
:100960008F83988749015A0167017801672B682BAB
:10097000692B09F494C0C501B4010E94762D2B01A6
:100980003C0120E030E0A901C501B4010E94232C04
:1009900087FF04C077FA709477F87094A7019601E6
:1009A000C701B6010E94BF2B69837A838B839C8326
:1009B0009B01AC01C301B2010E94272C2B013C0119
:1009C0006D817E818F8198850E94C22C9B01AC0134
:1009D000C301B2010E94232C40903001509031019C
:1009E000609032017090330120E030E0A90187FF70
:1009F00023C0C501B4010E94232C811107C0698165
:100A00007A818B819C810E94DD2D0DC0A50194010E
:100A1000C701B6010E94272C9B01AC015F77C5017D
:100A2000B4010E94BF2B6B017C01A30192010E94C3
:100A3000722D1816CCF12EC0C501B4010E94232CD2
:100A400081110DC069817A818B819C810E94DD2D8D
:100A50006B017C01F7FAF094F7F8F0940FC0A50150
:100A60009401C701B6010E94272C9B01AC015F775E
:100A7000C501B4010E94BE2B6B017C0177FA709412
:100A800077F87094A3019201C701B6010E94232C4C
:100A900087FD0AC05C2D4D2D3E2D2F2D09C050E045
:100AA00040E030E020E004C0542D452D362D272DA8
:100AB000652F742F832F922F28960FB6F894DEBFE0
:100AC0000FBECDBFDF91CF911F910F91FF90EF909F
:100AD000DF90CF90BF90AF909F908F907F906F905E
:100AE0005F904F900895CF92DF92EF92FF920F9315
:100AF0001F93CF93DF93EC018B016A0169E070E0F3
:100B000083ED93E00E94BB23EE24D7FCE094FE2CFF
:100B1000C017D107CCF4BE0183ED93E00E940224FC
:100B2000C701B6010E94E02421960C171D079CF70F
:100B300083ED93E0DF91CF911F910F91FF90EF90A4
:100B4000DF90CF900C94C123BE0183ED93E00E940F
:100B50000224C701B6010E94E0242197C017D107E3
:100B60009CF7E6CFCF93DF9390917B038091D203E4
:100B70009230C0F0882329F0C0914101D091420108
:100B800004C0C0913F01D091400186EA93E00E94E9
:100B90003231909342018093410143E050E0BC0127
:100BA000CE010CC081110CC06091410170914201D5
:100BB00043E050E080913F01909140010E94730515
:100BC00081E08093D203DF91CF910895CF93DF939B
:100BD00090917B038091D2039230C0F0882329F05A
:100BE000C0914101D091420104C0C0913F01D09118
:100BF000400186EA93E00E94323190934001809355
:100C00003F0143E050E0BC01CE010CC0882361F0FD
:100C100060913F017091400143E050E080914101BB
:100C2000909142010E9473051092D203DF91CF91FF
:100C3000089586EA93E00E9432318093180188E992
:100C400093E00E94323190931A0180931901089524
:100C5000AF92BF92CF92DF92EF92FF920F931F93CA
:100C60006E157F058007910734F42E153F05400768
:100C700051076CF10BC0E616F7060807190794F444
:100C8000A216B306C406D50624F106C0A216B30602
:100C9000C406D50614F116C02A153B054C055D05A2
:100CA000C4F419C06E157F058007910791F42A15C9
:100CB0003B054C055D057CF0A216B306C406D506BF
:100CC00064F007C02A153B054C055D0511F484E06E
:100CD00005C082E003C081E001C083E01F910F9155
:100CE000FF90EF90DF90CF90BF90AF9008958F92DC
:100CF0009F92AF92BF92CF92DF92EF92FF920F93AB
:100D00001F93CF93DF934B015C018A01BA018827BF
:100D100077FD8095982F0E94C22C2091CE033091B0
:100D2000CF034091D0035091D1030E94762DA501AD
:100D300094010E94272C6B017C0120E030E040E010
:100D400050E40E94722D87FD0AC0C701B6010E94BF
:100D50008F2CEB01633071050CF03FC002C0C1E085
:100D6000D0E067E571E08DE094E00E943F2822E04A
:100D700030E0B701A6018DE094E00E945D2A66EFA5
:100D800070E08DE094E00E940E2822E030E0B50192
:100D9000A4018DE094E00E945B2A6AEE70E08DE091
:100DA00094E00E940E284AE050E0B8018DE094E003
:100DB0000E94132965EE70E08DE094E00E940E28F9
:100DC0004AE050E0BE018DE094E00E941B2964EBF4
:100DD00070E08DE094E00E944C28CE01DF91CF912D
:100DE0001F910F91FF90EF90DF90CF90BF90AF9049
:100DF0009F908F9008958F929F92AF92BF92CF92C3
:100E0000DF92EF92FF92CF93DF935C01EB01BA0187
:100E1000882777FD8095982F0E94C22C6B017C015A
:100E2000B501882777FD8095982F0E94C22C4B0131
:100E30005C01BE01882777FD8095982F0E94C22C07
:100E40009B01AC01C501B4010E94272CA7019601AA
:100E50000E94762D9B01AC01C701B6010E94BE2BFA
:100E60004B015C010E948F2CEB01882777FD809558
:100E7000982F0E94C22C9B01AC01C501B4010E94B5
:100E8000BE2B20E030E040E05FE30E94722D181698
:100E90000CF42196CE01DF91CF91FF90EF90DF907F
:100EA000CF90BF90AF909F908F90089580911B013D
:100EB000882319F010921B01089581E080931B0193
:100EC00008958F929F92AF92BF92CF92DF92EF924E
:100ED000FF9269017A019B01AC010E94762D4B01C2
:100EE0005C01A7019601C701B6010E94762D9B0106
:100EF000AC01C501B4010E94BF2BFF90EF90DF90C1
:100F0000CF90BF90AF909F908F900C94DD2DCF939A
:100F1000DF9300D000D0CDB7DEB78091BE039091B3
:100F2000BF03A091C003B091C103892B8A2B8B2BE7
:100F300009F044C06091C2037091C3038091C4035F
:100F40009091C5030E94C22C9B01AC016091C60325
:100F50007091C7038091C8039091C90329833A8394
:100F60004B835C830E94C22C29813A814B815C8136
:100F70000E94610720E030E040E05FE30E94BF2B69
:100F80000E948F2C6093BE037093BF038093C003B5
:100F90009093C10368E970E08DE094E00E940E2810
:100FA0004091BE035091BF036091C0037091C10393
:100FB0002AE030E08DE094E00E9433296091BE0386
:100FC0007091BF038091C0039091C1030F900F9067
:100FD0000F900F90DF91CF9108958F929F92AF92D3
:100FE000BF92CF92DF92EF92FF924B015C016901B9
:100FF0007A016091C6037091C7038091C8039091F4
:10100000C9030E94C22CA50194010E94BE2B9B0122
:10101000AC010E94762D4B015C01A7019601C7012E
:10102000B6010E94762D9B01AC01C501B4010E945E
:10103000BF2BFF90EF90DF90CF90BF90AF909F902D
:101040008F900C94DD2D809124018823C1F16EE6F0
:1010500071E08DE094E00E943F2880E792E00E94DA
:10106000781E2091380130E040E050E00E94862E4A
:10107000BA01A9012AE030E08DE094E00E94C9287D
:101080006CEE71E08DE094E00E943F288CE292E0EB
:101090000E94781E2091380130E040E050E00E942C
:1010A000862EBA01A9012AE030E08DE094E00E948A
:1010B000C92867EE71E08DE094E00C945E280895F5
:1010C0004F925F926F927F928F929F92AF92BF9258
:1010D000CF92DF92EF92FF92CF93DF9300D000D0B8
:1010E000CDB7DEB74B015C0129013A016091C6031F
:1010F0007091C7038091C8039091C9030E94C22CCC
:101100006B017C019B01AC010E94762D69837A837F
:101110008B839C83A3019201C301B2010E94762DAF
:101120009B01AC0169817A818B819C810E94BE2BDD
:101130002B013C01A5019401C501B4010E94762D4B
:101140009B01AC01C301B2010E94BF2B4B015C01AA
:10115000A7019601C701B6010E94BF2B9B01AC01FC
:10116000C501B4010E94272C0F900F900F900F9093
:10117000DF91CF91FF90EF90DF90CF90BF90AF9035
:101180009F908F907F906F905F904F9008958F9277
:101190009F92AF92BF92CF92DF92EF92FF926B013C
:1011A0007C01CA01B9010E94762D4B015C01A701A7
:1011B0009601C701B6010E94762D9B01AC01C501C5
:1011C000B4010E94BE2BFF90EF90DF90CF90BF90B4
:1011D000AF909F908F900C94DD2D0F931F93CF9322
:1011E000DF938C01EB010E9409328883C8010196CC
:1011F0000E940932898382E090E0DF91CF911F91B4
:101200000F91089566E371E080E090E00E94ED08A0
:1012100080913601909137011816190634F08AE84A
:1012200092E0909337018093360167ED72E08DE094
:1012300094E00E940E2860913601709137014AE0D7
:1012400050E08DE094E00E941B2964E371E082E0AD
:1012500090E00E94ED0880913401909135011816BC
:10126000190634F08AE892E09093350180933401B6
:1012700068EC72E08DE094E00E940E2860913401E9
:10128000709135014AE050E08DE094E00C941B2908
:101290006FE371E08AE290E00E94ED0880913F01E7
:1012A000909140018936914030F08AE590E090932A
:1012B000400180933F0160E972E08DE094E00E947C
:1012C0000E2860913F01709140014AE050E08DE0AE
:1012D00094E00E941B2961E471E08CE290E00E949E
:1012E000ED0880914101909142018936914030F0A2
:1012F00084EB90E0909342018093410161E872E0B9
:101300008DE094E00E940E286091410170914201AD
:101310004AE050E08DE094E00C941B29EF92FF929C
:101320000F931F93CF93DF937C018B01C0E0D0E03C
:10133000CE018E0D9F1D0E940932F80181938F010D
:101340002196C430D105A1F784E090E0DF91CF91E0
:101350001F910F91FF90EF90089569E371E08EE087
:1013600090E00E948E0920E030E040E85FE3609169
:10137000390170913A0180913B0190913C010E94AA
:10138000232C87FF0CC080E090E0AEEBB2E48093AA
:10139000390190933A01A0933B01B0933C0167EB74
:1013A00072E08DE094E00E940E2840913901509146
:1013B0003A0160913B0170913C0122E030E08DE008
:1013C00094E00E945D2A6DE371E082E190E00E946A
:1013D000ED0880913D0190913E011816190634F0F8
:1013E00080E991E090933E0180933D0161EA72E0D3
:1013F0008DE094E00E940E2860913D0170913E01C5
:101400004AE050E08DE094E00C941B2960E371E029
:1014100086E190E00E948E09609130017091310167
:1014200080913201909133010E948F2C161617067D
:1014300064F080E090E0A8E4B4E4809330019093FD
:101440003101A0933201B09333016CE271E08AE183
:1014500090E00E948E0960912C0170912D01809185
:101460002E0190912F010E948F2C1616170664F002
:1014700080E090E0A8E4B4E480932C0190932D01E7
:10148000A0932E01B0932F0108958F929F92AF9257
:10149000BF92CF92DF92EF92FF920E9402090E94C8
:1014A000AD090E943D030E9448090E94060A65E2B8
:1014B00071E08EE190E00E948E0927E137EB41ED6B
:1014C00058E3609125017091260180912701909148
:1014D00028010E94232C87FF0CC08DEC9CECACE40F
:1014E000BFE38093250190932601A0932701B09339
:1014F00028018090390190903A01A0903B01B09072
:101500003C01A0913D01B0913E012091380130E0B5
:101510000E94BA2E0E94C22C6B017C019B01AC017F
:10152000C501B4010E94272C6093CE037093CF03B2
:101530008093D0039093D103A5019401C701B60114
:101540000E94272C6093CA037093CB038093CC0333
:101550009093CD0366E572E08DE094E00E940E2842
:101560004091CE035091CF036091D0037091D1038D
:1015700022E030E08DE094E00E945B2A66E472E0B5
:101580008DE094E00E940E284091CA035091CB0355
:101590006091CC037091CD0322E030E08DE094E0C7
:1015A0000E945B2A64E472E08DE094E00E944C2883
:1015B0006091360170913701882777FD8095982FCB
:1015C0000E94C22C2091CA033091CB034091CC03DE
:1015D0005091CD030E94762D0E948F2C6093C603FC
:1015E0007093C7038093C8039093C90368E272E0C5
:1015F0008DE094E00E940E284091C6035091C703ED
:101600006091C8037091C9032AE030E08DE094E056
:101610000E94C92866E272E08DE094E00E944C28A6
:101620006091340170913501882777FD8095982F5E
:101630000E94C22C2091CA033091CB034091CC036D
:101640005091CD030E94762D0E948F2C6093C2038F
:101650007093C3038093C4039093C5036EE172E05B
:101660008DE094E00E940E2868E072E08DE094E046
:101670000E940E284091C2035091C3036091C4039D
:101680007091C5032AE030E08DE094E00E94C92803
:1016900066E072E08DE094E00E940E288DE094E018
:1016A0000E9448281092BE031092BF031092C003FC
:1016B0001092C103FF90EF90DF90CF90BF90AF905A
:1016C0009F908F900895CF92DF92EF92FF9226E045
:1016D00040E051EE60E070E08DE094E00E94C926A9
:1016E00064E771E08DE094E00E945E2863E871E0B9
:1016F0008DE094E00E943F284AE050E061E070E015
:101700008DE094E00E941B296EE871E08DE094E08A
:101710000E945E280E94450A0E94D4024091300136
:1017200050913101609132017091330180E792E074
:101730000E941F2140912C0150912D0160912E019A
:1017400070912F0180E792E00E9484214091300146
:101750005091310160913201709133018CE292E03D
:101760000E941F2140912C0150912D0160912E016A
:1017700070912F018CE292E00E94842160912901F6
:1017800070912A01882777FD8095982F0E94C22C9E
:101790002091390130913A0140913B0150913C0137
:1017A0000E94272C6B017C0160913D0170913E01EC
:1017B000882777FD8095982F0E94C22C9B01AC0151
:1017C000C701B6010E94762D0E948F2C6B017C010F
:1017D000AB01BC0180E792E00E947E1EB701A6012A
:1017E0008CE292E00E947E1EE8E4F3E0119283E036
:1017F000EA37F807D9F70E94B8020E94B20564EFF1
:1018000071E080E090E0FF90EF90DF90CF900C943B
:10181000E024CF93DF93C0E0D0E060E0CE010E94EF
:1018200011322196C233D105C1F7DF91CF910C94CB
:10183000450A0F931F93CF93DF938C01EB016881CF
:101840000E9411326981C80101960E94113282E022
:1018500090E0DF91CF911F910F9108950F931F9307
:10186000CF93DF9300D000D000D0CDB7DEB786EAAB
:1018700093E00E9432318C019E838D8388E993E04E
:101880000E9432319C838B831A830983BE016F5F70
:101890007F4F80E090E00E94ED088D819E8129813C
:1018A0003A812817390749F00B973CF0BE016B5F6E
:1018B0007F4F80E090E00E94190CBE016F5F7F4F68
:1018C00082E090E00E94ED088B819C8129813A8121
:1018D0002817390749F00B973CF0BE016D5F7F4F29
:1018E00082E090E00E94190C0E94020926960FB631
:1018F000F894DEBF0FBECDBFDF91CF911F910F9146
:101900000895CF93DF9300D0CDB7DEB786EA93E09A
:101910000E9432319A838983BE016F5F7F4F82E1DB
:1019200090E00E94190C0E94450A0F900F90DF91E1
:10193000CF910895CF93DF9300D0CDB7DEB786EA7D
:1019400093E00E9432319A838983BE016F5F7F4F9B
:1019500084E190E00E94190C0E94450A0F900F90BC
:10196000DF91CF9108950F931F93CF93DF9300D012
:1019700000D0CDB7DEB786EA93E00E9432318C0109
:101980009C838B8388E993E00E9432319A83898318
:1019900020917B03233089F4BE016D5F7F4F8AE283
:1019A00090E00E94190CBE016F5F7F4F8CE290E0C7
:1019B0000E94190C0E94480937C02230A9F543E063
:1019C00050E0B8010E94730568EC70E080E090E0A0
:1019D0000E94E02469817A8143E050E08B819C8100
:1019E0000E94730568EC70E080E090E00E94E024C3
:1019F0006B817C8143E050E089819A810E9473056C
:101A000068EC70E080E090E00E94E02469817A81D7
:101A100043E050E08B819C810E94730568EC70E08C
:101A200080E090E00E94E0240F900F900F900F90C4
:101A3000DF91CF911F910F910895EF92FF920F9335
:101A40001F93CF93DF937C018B01C0E0D0E0F801BE
:101A500061918F01CE018E0D9F1D0E941132219642
:101A6000C430D105A1F784E090E0DF91CF911F91C0
:101A70000F91FF90EF900895CF93DF9300D000D0A7
:101A8000CDB7DEB786EA93E00E942E3169837A8370
:101A90008B839C83BE016F5F7F4F8EE090E00E943E
:101AA0001D0D0E94450A0F900F900F900F90DF912F
:101AB000CF91089586EA93E00E942E310E9414048B
:101AC00080917B03823061F488E993E00E94323197
:101AD000019731F460E371E086E190E00C941D0D14
:101AE000089586EA93E00E942E310E94420480917C
:101AF0007B03823061F488E993E00E9432310197E0
:101B000031F46CE271E08AE190E00C941D0D0895CF
:101B1000CF92DF92EF92FF9265E971E086ED93E05C
:101B20000E94642B83ED93E00E942123C090CA039E
:101B3000D090CB03E090CC03F090CD0360913601C0
:101B400070913701882777FD8095982F0E94C22CCD
:101B5000A70196010E94762D0E948F2C6093C603E8
:101B60007093C7038093C8039093C90360913401B5
:101B700070913501882777FD8095982F0E94C22C9F
:101B8000A70196010E94762D0E948F2C6093C203BC
:101B90007093C3038093C4039093C5036BE971E012
:101BA00088E393E00E94642B6FE971E082E393E0A5
:101BB0000E94642B63EA71E08CE293E00E94642B44
:101BC00067EA71E086E293E00E94642B6BEA71E0C1
:101BD00080E293E00E94642B6FEA71E08AE193E077
:101BE0000E94642B63EB71E084E193E00E94642B1C
:101BF00067EB71E08EE093E00E94642B6BEB71E089
:101C000088E093E00E94642B6FEB71E082E093E048
:101C10000E94642B63EC71E08CEF92E00E94642BD5
:101C200067EC71E086EF92E00E94642B6BEC71E050
:101C300080EF92E00E94642B6FEC71E08AEE92E0FC
:101C40000E94642B63ED71E084EE92E00E94642BAD
:101C500067ED71E08EED92E00E94642B6BED71E018
:101C600088ED92E00E94642B6FED71E082ED92E0CE
:101C70000E94642B63EE71E08CEC92E00E94642B76
:101C800060913D0170913E0141E080EC92E00E9444
:101C9000991A60913D0170913E0142E084EB92E01F
:101CA0000E94991A42E052E06CEF71E080E792E006
:101CB0000E94C5204EE052E068E072E08CE292E0C3
:101CC000FF90EF90DF90CF900C94C5208CEC92E0C9
:101CD0000E94F62A82ED92E00E94F62A88ED92E0B8
:101CE0000E94F62A8EED92E00E94F62A84EE92E09F
:101CF0000E94F62A8AEE92E00E94F62A80EF92E095
:101D00000E94F62A86EF92E00E94F62A8CEF92E07B
:101D10000E94F62A82E093E00E94F62A88E093E08F
:101D20000E94F62A8EE093E00E94F62A84E193E076
:101D30000E94F62A8AE193E00E94F62A80E293E06C
:101D40000E94F62A86E293E00E94F62A8CE293E053
:101D50000E94F62A82E393E00E94F62A88E393E049
:101D60000E94F62A86ED93E00C94F62A80E792E032
:101D70000E94CA1D8CE292E00E94CA1D81E08093FD
:101D8000420380E792E00E94781EAB01BC014C5FE9
:101D90005F4F6F4F7F4F80E792E00E945B228CE2A3
:101DA00092E00E94781EAB01BC014C5F5F4F6F4F09
:101DB0007F4F8CE292E00E945B2280E792E00E94DB
:101DC000781EAB01BC01445051096109710980E7DB
:101DD00092E00E945B228CE292E00E94781EAB01AE
:101DE000BC0144505109610971098CE292E00C94E4
:101DF0005B228F929F92AF92BF92CF92DF92EF922F
:101E0000FF9286EA93E00E9450319B01AC01C090A2
:101E10003801D12CE12CF12CC701B6010E94342EDF
:101E20004B015C0188E993E00E9450319B01AC01B9
:101E3000C701B6010E94342E6B017C01B501A401DB
:101E400080E792E00E947E1EB701A6018CE292E03C
:101E50000E947E1E0E94B60EFF90EF90DF90CF9002
:101E6000BF90AF909F908F900C94230880E792E0F2
:101E70000E94B11D8CE292E00E94B11D0E94B20549
:101E8000109242030895CF92DF92EF92FF920F9348
:101E90001F930E94B12400914303109144032091A9
:101EA00045033091460340911C01442359F1409170
:101EB0004203442339F16B017C01C01AD10AE20AC2
:101EC000F30A80911D0190911E01A0911F01B09114
:101ED00020018C159D05AE05BF05A4F46AE071E0F4
:101EE0008DE094E00E943F2866E171E08DE094E08F
:101EF0000E944C281F910F91FF90EF90DF90CF90A0
:101F00000C94360F1F910F91FF90EF90DF90CF90C0
:101F100008954F925F926F927F928F929F92AF92AD
:101F2000BF92CF92DF92EF92FF920F931F93CF93C6
:101F3000DF938C010E94B1244B015C01F80180E029
:101F400090E01192019682339105D9F7C12CD12CE2
:101F50007601C0E0D0E00E94B124209719F4C0E0DF
:101F6000D0E014C0DC01CB018C199D09AE09BF097A
:101F700085369105A105B1054CF0F80180E090E0AF
:101F80001192019682339105D9F7E9CF0E94430F50
:101F90000E94B124681979098A099B0920912101BD
:101FA000309122012901662457FC6094762C461654
:101FB00057066806790634F40E94B8020E94B124DC
:101FC0004B015C018DE094E00E94E625181619068D
:101FD00014F68DE094E00E94FF25F801EC0FFD1F40
:101FE0008A3011F08B3359F41082CF01801B910B92
:101FF000C19714F41192F9CF7724739403C08083AE
:102000002196712C0E94B1246B017C01772009F488
:10201000A2CF0E94B1240E94B12460934303709325
:102020004403809345039093460360933E0370936B
:102030003F03809340039093410381E0DF91CF9170
:102040001F910F91FF90EF90DF90CF90BF90AF90D6
:102050009F908F907F906F905F904F9008954F92D8
:102060005F926F927F928F929F92AF92BF92CF9228
:10207000DF92EF92FF92CF93DF9300D000D0CDB7E5
:10208000DEB72B013C0129833A834B835C830E949A
:10209000B12460934303709344038093450390936A
:1020A000460380E792E00E9427224B015C018CE20C
:1020B00092E00E9427226B017C0140E050E0BA01CF
:1020C00080E792E00E94A82140E050E0BA018CE253
:1020D00092E00E94A821C301B2010E94C22C0E947A
:1020E0008F2CAB01BC0180E792E00E940220698145
:1020F0007A818B819C810E94C22C0E948F2CAB0123
:10210000BC018CE292E00E94022080912B0181119F
:102110003DC080E792E00E94272220E030E0A90144
:102120000E94232C87FF04C0B7FAB094B7F8B0948C
:102130008CE292E00E94272220E030E0A9010E9478
:10214000232C87FF04C0F7FAF094F7F8F094B50158
:10215000A40180E792E00E94A821B701A6018CE2C9
:1021600092E00E94A82112C00E94430F8091230197
:10217000882361F080912B01882389F080E792E029
:102180000E9498208CE292E00E94982080E792E0E2
:102190000E94661E672B682B692B31F709C080E708
:1021A00092E00E9438228CE292E00E943822EECF28
:1021B0008CE292E00E94661E672B682B692BA1F6C9
:1021C0000F900F900F900F90DF91CF91FF90EF90B5
:1021D000DF90CF90BF90AF909F908F907F906F9047
:1021E0005F904F900C9423088F929F92AF92BF9272
:1021F000CF92DF92EF92FF92CF93DF9300D000D087
:10220000CDB7DEB786EA93E00E942E316B017C01E8
:102210006091380170E080E090E00E94C22C9B0148
:10222000AC01C701B6010E94762D6B017C0188E9E3
:1022300093E00E942E314B015C016091380170E007
:1022400080E090E00E94C22C9B01AC01C501B4016A
:102250000E94762D0E948F2C9B01AC01C701B60114
:1022600029833A834B835C830E948F2C29813A8196
:102270004B815C810F900F900F900F90DF91CF9169
:10228000FF90EF90DF90CF90BF90AF909F908F9096
:102290000C942F102F923F924F925F926F927F92E9
:1022A0008F929F92AF92BF92CF92DF92EF92FF9266
:1022B0000F931F93CF93DF93CDB7DEB7A0970FB6E1
:1022C000F894DEBF0FBECDBF2B013C01E982FA823C
:1022D0000B831C8384010E9460086D837E838F833F
:1022E0009887A30192010E94C70869877A878B8724
:1022F0009C87A601950169817A818B819C810E94CE
:1023000060082B013C0129813A814B815C810E944C
:10231000C7086B017C0120E030E040EA51E4C301D2
:10232000B2010E94722D18160CF003C26091C60310
:102330007091C7038091C8039091C90364517109DA
:10234000810991090E94C22C4B015C019B01AC01E7
:10235000C301B2010E94232C87FFEBC120E030E0D3
:1023600040EA51E4C701B6010E94722D18160CF024
:10237000E0C16091C2037091C3038091C403909146
:10238000C50364517109810991090E94C22C6983B6
:102390007A838B839C839B01AC01C701B6010E94A9
:1023A000232C87FFC6C120E030E040EA51E46D8174
:1023B0007E818F8198850E94722D18160CF0B9C10C
:1023C000A50194016D817E818F8198850E94232CC7
:1023D00087FFAFC120E030E040EA51E469857A85AB
:1023E0008B859C850E94722D18160CF0A2C1298144
:1023F0003A814B815C8169857A858B859C850E94B9
:10240000232C87FF96C1109224012D813E814F819C
:102410005885C301B2010E94BE2B4B015C01298586
:102420003A854B855C85C701B6010E94BE2B6B01C6
:102430007C0120E030E0A901C501B4010E94722DA9
:1024400024013501181624F077FA709477F8709407
:1024500020E030E0A901C701B6010E94722DA7015A
:10246000960118160CF05058C301B2010E94722D4B
:102470009801442737FD4095542F29833A834B8395
:102480005C831816E4F02601370177FA709477F828
:10249000709420E030E0A901C701B6010E94722DBE
:1024A00018162CF41C2D0D2DED86F98A04C0142D60
:1024B000052D6D86798A22242394312C3EC0240177
:1024C000350177FA709477F8709420E030E0A90134
:1024D000C501B4010E94722D18162CF4182D092D77
:1024E000AD86B98A04C0142D052D6D86798A222403
:1024F0002394312CB101882777FD8095982F0E9475
:10250000C22C9B01AC01612F702F8D8599890E948F
:10251000272C2B013C0169817A818B819C810E944F
:10252000C22C9B01AC01C301B2010E94722D18168E
:102530003CF53FEF231A330ADDCFB101882777FD41
:102540008095982F0E94C22C9B01AC01612F702FA7
:102550008D8599890E94272C2B013C0169817A8104
:102560008B819C810E94C22C9B01AC01C301B201F2
:102570000E94722D181624F44FEF241A340ADDCF6E
:10258000C101AA2797FDA095BA2F89839A83AB83AF
:10259000BC83BC01CD010E94C22C2B013C019B01DC
:1025A000AC01C501B4010E94272C6D877E878F87FF
:1025B000988BA3019201C701B6010E94272C698B59
:1025C0007A8B8B8B9C8B10922B01812C912C54013C
:1025D000C12CD12C76012D853E854F8558896D8182
:1025E0007E818F8198850E94BF2B6D837E838F8330
:1025F000988729893A894B895C8969857A858B8591
:102600009C850E94BF2B69877A878B879C879B015B
:10261000AC016D817E818F8198850E9461076D8BF1
:102620007E8B8F8B988F29853A854B855C856D8154
:102630007E818F8198850E94ED07698F7A8F8B8FBD
:102640009C8F20E030E040E850E460912C017091D4
:102650002D0180912E0190912F010E94762D2B014A
:102660003C01C701B6010E94C22C9B01AC016981EB
:102670007A818B819C81680D791D8A1D9B1D830148
:1026800072010E9496040E948F2C6B017C010E94B3
:10269000C22C2B013C01AB01BC0180E792E00E94FF
:1026A000A821B301A2018CE292E00E94A821698DC9
:1026B0007A8D8B8D9C8D0E948F2C9B01AC016D8936
:1026C0007E898F89988D2D8F3E8F4F8F58A30E94C2
:1026D0008F2C2D8D3E8D4F8D58A10E942F1091E093
:1026E000891A9108A108B108C101880D991D892B8B
:1026F00009F071CF81E08093240180932B01A09693
:102700000FB6F894DEBF0FBECDBFDF91CF911F9102
:102710000F91FF90EF90DF90CF90BF90AF909F9080
:102720008F907F906F905F904F903F902F900C9480
:10273000230861E171E08DE094E00E943F2865E2AA
:1027400071E08DE094E0A0960FB6F894DEBF0FBE66
:10275000CDBFDF91CF911F910F91FF90EF90DF9050
:10276000CF90BF90AF909F908F907F906F905F9031
:102770004F903F902F900C944C284F925F926F9205
:102780007F928F929F92AF92BF92CF92DF92EF9201
:10279000FF920F931F93CF93DF93CDB7DEB72C97A4
:1027A0000FB6F894DEBF0FBECDBF86EA93E00E945D
:1027B0002E316B017C016091380170E080E090E087
:1027C0000E94C22C9B01AC01C701B6010E94762D6C
:1027D0002B013C0188E993E00E942E316B017C01C2
:1027E000B09038018AE893E00E9432314C0180E7D2
:1027F00092E00E94781E69837A838B839C838CE2AB
:1028000092E00E94781E6D837E838F83988720E0FC
:1028100030E040EA51E4C301B2010E94232C87FD5D
:102820002EC06B2D70E080E090E00E94C22C9B01D6
:10283000AC01C701B6010E94762D5B016C0120E05E
:1028400030E040EA51E40E94232C87FD18C00E942A
:1028500087070E94C22C9B01AC01C301B2010E94F8
:10286000722D181664F00E9487070E94C22C9B01EB
:10287000AC01C601B5010E94722D181614F561E174
:1028800071E08DE094E00E943F286BE471E08DE000
:1028900094E02C960FB6F894DEBF0FBECDBFDF914B
:1028A000CF911F910F91FF90EF90DF90CF90BF904D
:1028B000AF909F908F907F906F905F904F900C940F
:1028C0004C286D817E818F8198850E94C22C9B014E
:1028D000AC0169817A818B819C8129873A874B87FA
:1028E0005C870E94C22C8301720129853A854B8541
:1028F0005C850E944A112C960FB6F894DEBF0FBE7D
:10290000CDBFDF91CF911F910F91FF90EF90DF909E
:10291000CF90BF90AF909F908F907F906F905F907F
:102920004F9008952F923F924F925F926F927F92B5
:102930008F929F92AF92BF92CF92DF92EF92FF92CF
:102940000F931F93CF93DF9300D000D0CDB7DEB7A6
:102950001701F80117FD3196F595E7954F01AA2467
:1029600097FCA094BA2C2B013C01481859086A081E
:102970007B086801EE24D7FCE094FE2CDA01C90143
:1029800088199909AA09BB094C015D0100E010E012
:10299000201631065CF1A701960160E070E0CB01E2
:1029A0000E94932A69837A838B839C83A701960173
:1029B00060E070E0CB010E94932A9B01442737FD21
:1029C0004095542F280D391D4A1D5B1DA981BA81E0
:1029D000BD01882777FD8095982F640D751D861D94
:1029E000971D0E942F100F5F1F4FD2CF0F900F9097
:1029F0000F900F90DF91CF911F910F91FF90EF906B
:102A0000DF90CF90BF90AF909F908F907F906F900E
:102A10005F904F903F902F9008954F925F926F92EA
:102A20007F928F929F92AF92BF92CF92DF92EF925E
:102A3000FF920F931F93CF93DF9300D000D0CDB7B9
:102A4000DEB786EA93E00E94503110913801C12E22
:102A5000D12CE12CF12C9B01AC01C701B6010E94E5
:102A6000342E4B015C0188E993E00E9450319B01B8
:102A7000AC01C701B6010E94342E2B013C018AE84B
:102A800093E00E943231212F30E0DC010E94BA2E07
:102A900069837A838B839C838CE793E00E94323135
:102AA0007C01609125017091260180912701909110
:102AB000280149815A810E947706AC016FEF70E0CE
:102AC000C7010E94FB067C0129813A81B901882750
:102AD00077FD8095982F0E94C22C2DEC3CEC4CE8A1
:102AE0005FE30E94762D0E948F2C8B01A30192013F
:102AF000C501B4010E9492140F900F900F900F9097
:102B0000DF91CF911F910F91FF90EF90DF90CF90C9
:102B1000BF90AF909F908F907F906F905F904F90FD
:102B20000895CF93DF93EC01AB01662757FD6095C5
:102B3000762F0E941920CE010E94661E672B682BFB
:102B4000692B51F00E94430F80912301882399F350
:102B5000CE010E949820EFCF0E94B12460934303DE
:102B6000709344038093450390934603DF91CF9184
:102B700008958F929F92AF92BF92CF92DF92EF9281
:102B8000FF920F931F93CF93DF935C01EB016A01D8
:102B90004901E114F10499F564EA70E08DE094E0F4
:102BA0000E944C2880911B01882349F0D7FE03C066
:102BB0008FEFC81AD80AB601759567950BC0D7FE76
:102BC00003C08FEFC81AD80AB6017595679571953D
:102BD00061957109CE010E949115B401C5010E9451
:102BE0009115DF91CF911F910F91FF90EF90DF90A2
:102BF000CF90BF90AF909F908F900C94560780918C
:102C00001B01E016F10629F5882349F057FF03C0A0
:102C10008FEFC81AD80AB601759567950BC057FF94
:102C200003C08FEFC81AD80AB601759567957195DC
:102C300061957109CE01DF91CF911F910F91FF90A6
:102C4000EF90DF90CF90BF90AF909F908F900C94BB
:102C50009115882311F0BA01BDCF66277727641B31
:102C6000750BB8CF2F923F924F925F926F927F92E7
:102C70008F929F92AF92BF92CF92DF92EF92FF928C
:102C80000F931F93CF93DF93CDB7DEB727970FB680
:102C9000F894DEBF0FBECDBF1B015F834E83298337
:102CA000141615060CF078C0BA010E94502E7B83D2
:102CB0006A83BC01882777FD8095982F0E94C22CDB
:102CC0004B015C012E813F81B901882777FD8095FA
:102CD000982F0E94C22C9B01AC01C501B4010E9437
:102CE000272C2B013C01C12CD12C812C912C54017F
:102CF0008A819B8101969D838C83A3019201C501EA
:102D0000B4010E94BF2B4B015C0120E030E040E8A1
:102D10005FE30E94722D87FD0DC020E030E040E8A7
:102D20005FE3C501B4010E94BE2B4B015C012C8105
:102D30003D8102C02A813B819981923049F0E9812D
:102D4000E330A9F0F981F43061F43195219531092E
:102D500076010E811F81A1016CE272E080E792E0B2
:102D60000EC08981813069F4319521953109760150
:102D70000E811F81A10160E772E08CE292E00E9467
:102D8000B9150E9423089FEFC91AD90AEE81FF8165
:102D9000EC15FD050CF0B1CF27960FB6F894DEBF09
:102DA0000FBECDBFDF91CF911F910F91FF90EF909C
:102DB000DF90CF90BF90AF909F908F907F906F905B
:102DC0005F904F903F902F9008952F923F924F9297
:102DD0005F926F927F928F929F92AF92BF92CF92AB
:102DE000DF92EF92FF920F931F93CF93DF93CDB7B4
:102DF000DEB72A970FB6F894DEBF0FBECDBF86EAC6
:102E000093E00E945031B0903801CB2CD12CE12CB2
:102E1000F12C9B01AC01C701B6010E94342E2B019D
:102E20003C0188E993E00E9450319B01AC01C7014D
:102E3000B6010E94342E69837A838B839C838AE84F
:102E400093E00E9432312B2D30E0DC010E94BA2E3B
:102E50006D837E838F8398878CE793E00E94323165
:102E60009A8789878D809E8097FE03C00FEF801A16
:102E7000900A95948794C401880F991F2D803E80F5
:102E8000281A390A809118018130C9F48CE292E045
:102E90000E94781E5B016C0180E792E00E94781E20
:102EA0007B018C0129813A814B815C81C301B20194
:102EB0000E94280690E090931A01809319012091B6
:102EC000190130911A016401EE24D7FCE094FE2C24
:102ED000C101AA2797FDA095BA2F22303105A9F488
:102EE000B301A2014C195D096E097F09C40CD51C00
:102EF000E61CF71C89809A80AB80BC802A013B01CC
:102F0000480E591E6A1E7B1E54C023303105C9F479
:102F100049815A816B817C814C195D096E097F0959
:102F200089809A80AB80BC808C0C9D1CAE1CBF1C21
:102F3000730162018A019B01080F191F2A1F3B1FA1
:102F400034C024303105C9F4B301A2014C0D5D1D1C
:102F50006E1D7F1D930182010C191D092E093F0969
:102F60006801790189809A80AB80BC802A013B018D
:102F7000481A590A6A0A7B0A1CC049815A816B8126
:102F80007C814C0D5D1D6E1D7F1D89809A80AB80FC
:102F9000BC808C189D08AE08BF08730162018A01CD
:102FA0009B01081B190B2A0B3B0B09831A832B83EC
:102FB0003C836091250170912601809127019091B9
:102FC00028014D815E810E947706AC016FEF70E0B1
:102FD00089859A850E94FB061C0129813A814B81D3
:102FE0005C81C301B2010E942F1012E0211631044E
:102FF00044F020911901A1016D817E81CB010E94D5
:103000003216A5019401C701B6012A960FB6F894AD
:10301000DEBF0FBECDBFDF91CF911F910F91FF900B
:10302000EF90DF90CF90BF90AF909F908F907F9068
:103030006F905F904F903F902F900C942F103F9285
:103040004F925F926F927F928F929F92AF92BF92B8
:10305000CF92DF92EF92FF920F931F93CF93DF9364
:10306000CDB7DEB72A970FB6F894DEBF0FBECDBF3F
:1030700086EA93E00E9432312091380130E0DC0191
:103080000E94BA2E6B017C017A87698788E993E0F8
:103090000E942E314B015C018AE893E00E942E31A0
:1030A00069837A838B839C838CE793E00E942E3123
:1030B0006D837E838F8398873090180182E08093A0
:1030C00018014090250150902601609027017090D2
:1030D000280100E010E029813A814B815C81C50123
:1030E000B4010E94232C181614F10F5F1F4F809219
:1030F000250190922601A0922701B09228014985CE
:103100005A85C501B4010E94770622E0AC016985A9
:103110007A85CB010E9432162D813E814F815885E0
:10312000C501B4010E94BF2B4B015C01D4CF40927A
:103130002501509226016092270170922801AA244D
:10314000BB24AC18BD08B5018CE292E00E94911539
:10315000C60129853A8537FD01969595879588247E
:103160009924881A990AC601D7FC01967C01F59426
:10317000E794CC24C394D12C0C151D059CF0B4010C
:103180008CE292E00E949115B50180E792E00E94E6
:103190009115B7018CE292E00E9491153FEFC31A9E
:1031A000D30AEACF4092250150922601609227016E
:1031B00070922801309218012A960FB6F894DEBF5B
:1031C0000FBECDBFDF91CF911F910F91FF90EF9078
:1031D000DF90CF90BF90AF909F908F907F906F9037
:1031E0005F904F903F900895CF93DF93EC0168E399
:1031F00073E00E949E2B882319F00E94F410B3C044
:103200006CEF72E0CE010E949E2B882319F00E9481
:10321000BD13A9C062E373E0CE010E949E2B8823F8
:1032200019F00E9470049FC068ED72E0CE010E9408
:103230009E2B882319F00E945A0D95C062ED72E012
:10324000CE010E949E2B882319F00E94710D8BC025
:103250006CE273E0CE010E949E2B882319F00E943D
:10326000E51681C066E273E0CE010E949E2B8823A2
:1032700019F00E940D1577C060E273E0CE010E9444
:103280009E2B882319F00E9419066DC06AE173E035
:10329000CE010E949E2B882319F00E941F1863C044
:1032A00064E173E0CE010E949E2B882319F00E94F6
:1032B000F90E59C06EE073E0CE010E949E2B882368
:1032C00019F00E94E6054FC068E073E0CE010E944D
:1032D0009E2B882319F00E94B20545C062E073E07E
:1032E000CE010E949E2B882319F00E94B30C3BC094
:1032F00066EF72E0CE010E949E2B882319F00E9497
:103300002E0C31C064EE72E0CE010E949E2B882309
:1033100019F00E943C0D27C06EED72E0CE010E94B4
:103320009E2B882319F00E94810C1DC06CEC72E06A
:10333000CE010E949E2B882319F00E949A0C13C084
:1033400060EF72E0CE010E949E2B882319F00E944C
:10335000540309C06AEE72E0CE010E949E2B8823BE
:1033600021F00E94090C81E001C080E0DF91CF9143
:103370000895CF93DF93EC010E94F418811107C0E8
:10338000CE010E94BE02DF91CF910C94B802DF9172
:10339000CF9108950F931F93CF93DF9300D000D068
:1033A00000D0CDB7DEB78C010E94A0028823D9F0EF
:1033B00068E473E0CE0101960E94642BCE01019671
:1033C0000E94B919CE0101960E94F62AF80180E008
:1033D00090E01192019682339105D9F7109247033C
:1033E0000E94B80217C061E171E08DE094E00E9494
:1033F0003F286AE073E08DE094E00E940E28B80157
:103400008DE094E00E943F286CEF72E08DE094E044
:103410000E944C2810927B0326960FB6F894DEBFCC
:103420000FBECDBFDF91CF911F910F91089588E41A
:1034300093E00E94890F882321F088E493E00C94A4
:10344000CA19089584B5836884BD17BC61E086E01D
:103450000C94772584B5836284BD18BC61E085E057
:103460000C947725CF93DF9360E08CE00E94B02529
:1034700060E088E00E94B025C7E0D0E060E084E032
:103480000E94B0258091DD0390E00C2E02C095953E
:1034900087950A94E2F780FF02C061E001C060E016
:1034A00088E00E94B02561E084E00E94B025219769
:1034B00028F761E08CE0DF91CF910C94B025CF9399
:1034C000DF93EC0161E08CE00E94772561E087E00A
:1034D0000E94772561E088E00E94772561E084E022
:1034E0000E9477251092DD03CE010E94321A60E01F
:1034F00087E0DF91CF910C94B025E0EBF0E0908174
:103500009368908387708093B1001092B30061E05C
:103510008BE00C947725E0EBF0E090819362908350
:1035200087708093B1001092B40061E083E00C9446
:103530007725EF92FF920F931F93CF93DF931F9204
:10354000CDB7DEB77C018B018CED93E049830E94FF
:103550005F1AF7011183008349814283138641304A
:1035600029F58091DD03817E8093DD038CED93E06E
:103570000E94321A61E08BE00E94772561E083E0CF
:103580000E94772561E08BE00E94B02561E083E036
:103590000E94B02581E00E947D1A81E00E948B1A72
:1035A0008FEF8093B3008093B40022C0423001F5C6
:1035B0008091DD038E718093DD038CED93E00E949A
:1035C000321A61E085E00E94772561E086E00E9482
:1035D000772561E085E00E94B02561E086E00E94E9
:1035E000B0250E94221A0E942A1A8FEF87BD88BD3B
:1035F0000F90DF91CF911F910F91FF90EF90089561
:103600000F931F93CF93DF93EC017A81713041F0D8
:10361000723009F0C4C0B0E4A0E831E020E204C098
:10362000B0E1A8E032E024E08B85413019F483FF5B
:1036300005C00DC0423049F483FF09C0613011F468
:10364000805F01C080518B8741C0433031F46130CD
:1036500011F4885FF8CF8850F6CF4430B9F5613067
:1036600011F48F5F01C081508B875B855F735B872F
:10367000852F90E0503148F4E3E5F1E0E81BF90BC9
:103680005081FC01ED5BFE4F1FC060EF650F6031A4
:1036900038F4FC01ED5CFE4F5081E3E6F1E012C02E
:1036A0005052503148F4E3E7F1E0E81BF90B508148
:1036B000FC01ED5DFE4F08C0FC01ED5EFE4F508148
:1036C000E3E8F1E0E81BF90B808102C05FEF8FEFC8
:1036D0009B859F739B87713029F45093B30080932F
:1036E000B40004C0723011F457BD88BD132F122BE3
:1036F0000B2F0A2B802F812B80959091DD0389233E
:103700008093DD039B85443001F5903118F4812BC3
:103710008093DD0380EF890F803130F43A2B809164
:10372000DD03832B8093DD0380EE890F803128F445
:103730008091DD03802B8093DD039053903148F519
:103740002B2B8091DD03822B0EC0492F4695469589
:10375000469550E048305105E0F44C5C5F4FFA016B
:103760000C94A52E812B8093DD0313C03A2B382BAC
:103770003093DD030EC0A82BA093DD030AC0802B7D
:10378000F2CFB82BB093DD0304C02B2B282B209352
:10379000DD038CED93E00E94321A8B8501C080E03E
:1037A000DF91CF911F910F9108951092DC0308953E
:1037B0000F931F93DC0112960C9110E00930110554
:1037C000C0F5F801E45CFF4F0C94A52EDC01ED91EF
:1037D000FC910084F185E02D29C0DC01ED91FC9184
:1037E0000284F385E02D22C0DC01ED91FC9104847C
:1037F000F585E02D1BC0DC01ED91FC910684F78579
:10380000E02D14C0DC01ED91FC910088F189E02DE0
:103810000DC0DC01ED91FC910288F389E02D06C01A
:10382000DC01ED91FC910488F589E02D1F910F9149
:1038300009941F910F910895CF93DF93EC01CB0171
:10384000BA0126E030E040E050E00E94862E62306F
:1038500071058105910559F18CF46115710581059A
:103860009105F1F06130710581059105C1F5E8819F
:10387000F9810480F581E02D65E02DC0643071058B
:103880008105910511F1D4F065307105810591052F
:1038900031F5E881F9810480F581E02D66E01BC0F7
:1038A000E881F9810480F581E02D64E014C0E881AD
:1038B000F9810480F581E02D61E00DC0E881F98196
:1038C0000480F581E02D63E006C0E881F981048081
:1038D000F581E02D62E0CE01DF91CF910994DF9177
:1038E000CF910895CF93DF934770552766277727A9
:1038F00041505109DC01CD91DC914730510528F44C
:103900004B5B5F4FFA010C94A52EEC81FD8161E0C9
:103910001BC0EC81FD8165E017C0EC81FD8164E096
:1039200013C0EC81FD8166E00FC0EC81FD8162E097
:103930000BC0EC81FD816AE007C0EC81FD8168E08D
:1039400003C0EC81FD8169E0DF91CF910994AF92D2
:10395000BF92DF92EF92FF920F931F93CF93DF936B
:103960001F92CDB7DEB78C01FC018281843041F01B
:10397000883031F0833031F0863021F022E003C00E
:1039800024E001C023E0A12CB12CE62EF12CDD2493
:10399000D394F801EA0DFB1DC7010A2C02C09595CE
:1039A00087950A94E2F7678180FD6D2583812983DD
:1039B0000E94B025FFEFAF1ABF0A2981A21648F373
:1039C0000F90DF91CF911F910F91FF90EF90DF90BB
:1039D000BF90AF9008950F931F93CF93DF93EC01A7
:1039E000E881F9810480F581E02D8C010D5B1F4F8A
:1039F000D8018C91882311F062E001C060E0CE0113
:103A00000995E881F9810480F581E02DD8018C9138
:103A1000882311F063E001C061E0CE0109958BA518
:103A20009CA50E940825E881F9810480F581E02D9C
:103A3000D8018C91882311F062E001C060E0CE01D2
:103A4000DF91CF911F910F910994CF93DF93EC01F8
:103A500020E030E0A9016B897C898D899E890E94D4
:103A6000722D18161CF4EFA5F8A902C0E9A9FAA94D
:103A7000DF91CF9109944370552766277727DC01A2
:103A8000ED91FC910480F581E02D423051056105F6
:103A9000710571F0433051056105710559F04130F0
:103AA00051056105710511F062E005C063E003C0D6
:103AB00061E001C060E00994CF93DF93EC01CB019A
:103AC000BA0123E030E040E050E00E94862E6130F1
:103AD00071058105910581F06230710581059105BF
:103AE00091F0672B682B692BC1F4E881F981048080
:103AF000F581E02D64E00DC0E881F9810480F58155
:103B0000E02D61E006C0E881F9810480F581E02DB7
:103B100062E0CE01DF91CF910994DF91CF910895BA
:103B20004370552766277727DC01ED91FC910480CF
:103B3000F581E02D423051056105710571F043308A
:103B400051056105710559F0413051056105710557
:103B500011F065E005C066E003C06AE001C069E0FD
:103B60000994CF93DF93EC018A81882381F0E88167
:103B7000F9810480F581E02D60E0CE0109958EA5E4
:103B80008F3F29F06DA5DF91CF910C94B025DF9187
:103B9000CF910895CF93DF93EC018A81882351F16F
:103BA00061E08B810E94772561E08C810E947725FE
:103BB0008A81843011F0883039F461E08D810E946F
:103BC000772561E08E8106C0833011F0863021F4C4
:103BD00061E08D810E9477258EA58F3F59F061E0CD
:103BE0000E9477256DA581E068278EA5DF91CF9192
:103BF0000C94B025DF91CF910895CF92DF92EF9290
:103C0000FF920F931F93CF93DF93EC014BA15CA125
:103C10006DA17EA1452B462B472B09F44DC00E9478
:103C2000BD246B017C010FA118A529A53AA54BA1C4
:103C30005CA16DA17EA1400F511F621F731F401731
:103C400051076207730730F0C416D506E606F7067B
:103C500058F405C0C416D506E606F70668F1C01686
:103C6000D106E206F30640F5FE01ED5BFF4F8081D1
:103C70004B855C856D857E85882329F04F5F5F4F7E
:103C80006F4F7F4F04C041505109610971094B8743
:103C90005C876D877E87E881F9814B855C856D85C2
:103CA0007E850680F781E02DCE010995CFA2D8A6AA
:103CB000E9A6FAA681E001C080E0DF91CF911F91D3
:103CC0000F91FF90EF90DF90CF9008950F931F9387
:103CD000FC01678570898189928903851485258512
:103CE0003685601B710B820B930B1F910F9108950A
:103CF000FC0163857485858596850895FC0143875D
:103D00005487658776874787508B618B728B13AAA0
:103D100014AA15AA16AA13A214A215A216A20895EF
:103D20002F923F924F925F926F927F928F929F92CB
:103D3000AF92BF92CF92DF92EF92FF920F931F93B9
:103D4000CF93DF9300D000D0CDB7DEB71C01FC01CC
:103D500087849088A188B28883859485A585B68557
:103D6000881A990AAA0ABB0A63897489858996897F
:103D70009B01AC010E94762D6B017C01F101638DEA
:103D8000748D858D968D9B01AC010E94BF2B9B018C
:103D9000AC01C701B6010E94272C0E948F2C811410
:103DA0009104A104B104A1F462307105810591056B
:103DB0000CF07CC0F10113A214A215A216A2138A62
:103DC000148A158A168A13AA14AA15AA16AA03C158
:103DD000F10103A914A925A936A9ED5BFF4F181419
:103DE00019041A041B04FCF410161106120613061B
:103DF0004CF4681579058A059B054CF52081211145
:103E000055C025C0011511052105310509F44EC025
:103E1000681579058A059B050CF048C080818823C8
:103E200009F444C037C01016110612061306F4F444
:103E3000002711279801081919092A093B09601759
:103E40007107820793071CF42081222379F19B01DB
:103E5000AC0188279927DC01821B930BA40BB50BBF
:103E6000F10183AB94ABA5ABB6AB20C00115110536
:103E700021053105D9F0CC24DD247601C818D908F4
